:1000000002010A02012A0000000000320000000084
:10001000000000320000000000000032000000007C
:100020000000003200000000000000000000C39546
:10003000F02212002E60044002E422740122C0E08B
:10004000740A1470FDD0E0002274C811551155D502
:10005000E0F9D8F522C0E07419113E1470FBD0E02D
:10006000220022D2B01161D2B111617F0AD330B027
:100070000C30B109DFF8C2B11161C2B0C3920422E1
:10008000C2B11161D2B01161D2B12292B1116150ED
:100090000C7F0A20B107DFFBD2B0D38013D2B0119E
:1000A000617F0A20B007DFFBD2B1D38003C2B0C3A7
:1000B00022D2B11161D2B011617F0A20B005DFFBFD
:1000C000D38007A2B192D5C2B0C3227E0833118B70
:1000D000400CDEF911B14006A2D550021180920405
:1000E0002233FD7E0811B1400CA2D533DEF7CD13CB
:1000F000CD118BD2B1920422F874E204000000000A
:100100000000000070F500D8F022787FE4F6D8FDFA
:1001100075812A752000C2B4C2B3C295C294D2B50B
:10012000D2AFD2A8438702020124C0D0C2D3C0E01C
:10013000C0F0C083C082C000C001C002C003C004C0
:10014000C005C006C007C008C009C00AC00BC00C6B
:10015000C00DC00EC00FC010C011746411F8A2B25F
:100160009204500302019BC2B5742811F8D294D2B4
:1001700095740A11F8C295740A11F8C294D2957454
:100180000A11F8C295A2979204500302019031CE51
:10019000A2979204400302019B519ED011D010D02F
:1001A0000FD00ED00DD00CD00BD00AD009D008D073
:1001B00007D006D005D004D003D002D001D000D0A3
:1001C00082D083D0F0D0E0D0D0322202015A752202
:1001D0000175F00FE52211327003020283752100D0
:1001E00075230075F007E5231132700302022275B2
:1001F000F002E521A4C0E07821D0E0F6E4A29692D6
:10020000E0F5288528F0E52125F0C0E07821D0E050
:10021000F6D295740111F8C2950523E52360030217
:1002200001E3A2919204500302023FE4A29092E003
:10023000F5298529F07410A4C0E07824D0E0F6A256
:10024000919204400302026AE4A29092E0F52985AB
:1002500029F07410A4C0E07824D0E0F675F020E511
:100260002425F0C0E07824D0E0F68522F0E52425AE
:10027000F0C0E07824D0E0F671D10522E5226003D9
:100280000201D1C295C294D2B57525FF75270171BF
:10029000ACA2B29204500302029D02029122752286
:1002A0000175F00FE522113270030203647521001D
:1002B00075230075F007E523113270030202EE7515
:1002C000F002E521A4C0E07821D0E0F6E4A2969205
:1002D000E0F5288528F0E52125F0C0E07821D0E080
:1002E000F6D295C2950523E52360030202B3852269
:1002F0002471E6E521B526030202FE020301020392
:100300005B75F010E52225F0C0E07824D0E0F671AE
:10031000E6E521B5260302031C02031F02035B75F9
:10032000F020E52225F0C0E07824D0E0F671E6E583
:1003300021B5260302033A02033D02035B75F03048
:10034000E52225F0C0E07824D0E0F671E6E521B59D
:10035000260302035802039102035B0522E5226093
:10036000030202A1C295C294D2B5D2B57525FF751C
:10037000270171ACA2B292045003020380020374FD
:1003800078011149D2B478021149C2B478011149F7
:1003900022C295C294D2B575255A75270971ACA2AF
:1003A000B2920450030203AB02039F227522008520
:1003B00027F0E522113270030203D0D2B3E52511F4
:1003C000F8C2B3E52511F80522E52260030203AF68
:1003D00022116374A011CBE52411CBE52111CB11BF
:1003E00080740A11F822116374A011CBE52411CB9B
:1003F000116374A111CBD311E1F5F085F0261180C2
:1004000022000000000000000000000000000000CA
:00000001FF
